:020000040000FA
:040000006A303A2800
:08000800A000030EA100831209
:100010008B1C32288B1031181428B11C3228643004
:10002000010203183128182800001628172818285C
:1000300019281A281B281C281D281E281F283110A3
:10004000B114A810031005190314AA0DA90DA80DC9
:10005000B00B322831152A08AF002908AE00280855
:10006000AD00B11081010B11210E8300A00E200EF6
:02007000090085
:0C007400203084008001840A80300402E7
:10008000031C3C281230B000582283160C30850522
:1000900087018312850187010730990000309A009B
:1000A000103083168E008312603083168F00831207
:1000B0000030831691009F008312C83083168100A0
:1000C000831231309000003083168C008312103080
:1000D0008B00BC1B6D28851D7C233C1C70280623CF
:1000E000831620309B001C141A088312C1000130B3
:1000F000C1080319C10081018E018F010B118B1002
:100100000B108C018B1793203119A9203522B30BCA
:100110009128031085190314B90DF0303902031921
:10012000C4211B2383286400311808000B1D08001C
:100130000B11B11031141230B000051DA428321477
:1001400083160113831208003210831601178312DD
:10015000080031110130B7008B13203037078316A8
:100160009B001C141A088312A400A500C030A50629
:100170001030370783169B001C141A088312A30043
:100180000030370783169B001C141A088312A20044
:100190008B17321CD12822090339A200A309A40914
:1001A000A50922082D02031DBE2923082E02031DC6
:1001B000BE2924082F02031D4B2901303702031DDD
:1001C000E8283C19E7283D18E8283D143E14702221
:1001D00002303702031DF3283C19F228BD18F3281A
:1001E000BD143E14772203303702031DFE283C194C
:1001F000FD283D19FE283D153E147E2204303702AD
:10020000031D09293C190829BD190929BD153E14EA
:10021000852205303702031D14293C1913293D1A84
:1002200014293D163E148C2206303702031D1F2967
:100230003C191E29BD1A1F29BD163E1493220730F2
:100240003702031D2A293C1929293D1B2A293D175C
:100250003E149A2208303702031D35293C193429EF
:10026000BD1B3529BD173E14A12209303702031DDD
:1002700040293C193F294218402942143E14A82223
:100280000A303702031D4B293C194A29C2184B2951
:10029000C2143E14AF2225082F02031DBE290130CF
:1002A0003702031D5A293C1959293D1C5A293D1072
:1002B0003E14B62202303702031D65293C19642919
:1002C000BD1C6529BD103E14BA2203303702031D40
:1002D00070293C196F293D1D70293D113E14BE2225
:1002E00004303702031D7B293C197A29BD1D7B2967
:1002F000BD113E14C22205303702031D86293C1968
:1003000085293D1E86293D123E14C622063037023D
:10031000031D91293C199029BD1E9129BD123E143F
:10032000CA2207303702031D9C293C199B293D1F17
:100330009C293D133E14CE2208303702031DA72905
:100340003C19A629BD1FA729BD133E14D22209308E
:100350003702031DB2293C19B129421CB2294210AF
:100360003E14D6220A303702031DBD293C19BC2990
:10037000C21CBD29C2103E14DA22BE29B70A0B30B6
:10038000370203180800AC280130B600B300B400EF
:10039000B500B70085018701B1139320B30B042A80
:1003A000031085190314B90DF030390203192B2AF3
:1003B000B40B042A013037020319DE22023037025F
:1003C0000319E222033037020319E6220430370210
:1003D0000319EA22053037020319EE2206303702EC
:1003E0000319F222073037020319F62208303702C8
:1003F0000319FA22093037020319FE220A303702A4
:10040000031902239630B400311DCD293111321C5D
:100410000E2A2D090339AD00AE09AF092F1CB11307
:100420002F1CCD29B11BCD292E18CD29B1178B1327
:1004300020303707BB002F08BA004322103037079F
:10044000BB002E08BA00432200303707BB002D083E
:10045000BA0043228B1785018701B70AB6010B301A
:100460003702031CCD29062308003E1C08003E105D
:100470001030BB003D08BA0043223030BB004208B8
:10048000BA00432208008B133A0883161C159A0001
:1004900083123B0883169B0055309D00AA309D00B7
:1004A0009C1464009C18512A1C1183128B1708009D
:1004B000831600309B001C141A088312BC003C1CDD
:1004C0000800831610309B001C141A088312BD000C
:1004D000831630309B001C141A088312C2000800D7
:1004E000051640084107D0000F08D1000800851606
:1004F00040084107D2000F08D30008000514400847
:100500004107D4000F08D5000800851440084107B2
:10051000D6000F08D7000800871440084107D8000C
:100520000F08D9000800071540084107DA000F0836
:10053000DB000800071440084107DC000F08DD005D
:100540000800871640084107DE000F08DF0008009A
:10055000071640084107CC000F08CD00080087159A
:1005600040084107CE000F08CF00080005128E0199
:100570008F01080085128E018F01080005108E0181
:100580008F01080085108E018F01080087108E01F1
:100590008F01080007118E018F01080007108E01DE
:1005A0008F01080087128E018F01080007128E014B
:1005B0008F01080087118E018F0108000508103A8D
:1005C000850008000508203A850008000508013A62
:1005D000850008000508023A850008000708023A6D
:1005E000870008000708043A870008000708013A56
:1005F000870008000708203A870008000708103A1B
:10060000870008000708083A870008003D1805160B
:10061000BD1885163D190514BD1985143D1A87149A
:10062000BD1A07153D1B0714BD1B87164218071678
:10063000C218871508003C1D080050084002031D21
:10064000262B51080F02031C262B051252084002CC
:10065000031D2F2B53080F02031C2F2B8512540848
:100660004002031D382B55080F02031C382B0510C0
:1006700056084002031D412B57080F02031C412B53
:10068000851058084002031D4A2B59080F02031C0D
:100690004A2B87105A084002031D532B5B080F0298
:1006A000031C532B07115C084002031D5C2B5D08E3
:1006B0000F02031C5C2B07105E084002031D652B14
:1006C0005F080F02031C652B87124C084002031DB4
:1006D0006E2B4D080F02031C6E2B07124E084002B2
:1006E000031D772B4F080F02031C772B87110C1C5F
:1006F00008000C10C00A0800B601B301B4013C1C8C
:10070000842BBC01BC148B2BBC1C892BBC013C155D
:100710008B2BBC013C143C08B60064008F2B902B43
:10072000912B922B932BB41B0516B41F0512B30B00
:100730008D2BB40B8D2B0310B60CB608031D8D2B1F
:0C0740000030BB003C08BA004322080057
:084000000900030005000500A2
:02400E00CC33B1
:10420000010003000300030003000200020002009B
:1042100002000000000000000000FF00FF00FF009F
:10422000000000000000000000000000000000008E
:104230000000C000C000C000C000FF00FF00FF0081
:104240000100C300F300CF00FF00C300F300CF0064
:10425000FF00C300F300CF00FF00FF00FF00FF00DE
:10426000FF00FF00FF00FF00FF00FF00FF00FF0056
:10427000FF00FF00FF00FF00FF00FF00FF00FF0046
:10428000FF00FF00FF00FF00FF00FF00FF00FF0036
:10429000FF00FF00FF00FF00FF00FF00FF00FF0026
:1042A000FF00FF00FF00FF00FF00FF00FF00FF0016
:1042B000FF00FF00FF00FF00FF00FF00FF00FF0006
:1042C000FF00FF00FF00FF00FF00FF00FF00FF00F6
:1042D000FF00FF00FF00FF00FF00FF00FF00FF00E6
:1042E000FF00FF00FF00FF00FF00FF00FF00FF00D6
:1042F000FF00FF00FF00FF00FF00FF00FF00AA001B
:00000001FF
